:100000003BC0AEC154C053C052C051C050C04FC01D
:100010004EC04DC04CC04BC04AC049C048C047C08C
:1000200046C045C044C009021200010100A01909E0
:10003000040000000000000012011001FF00000891
:10004000C016DC050401010200010E035500530037
:1000500042006100730070001C0377007700770096
:100060002E00660069007300630068006C002E00BB
:10007000640065000403090411241FBECFE5D4E029
:10008000DEBFCDBF10E0A0E6B0E0EAEAF5E102C0D5
:1000900005900D92A636B107D9F720E0A6E6B0E0AC
:1000A00001C01D92A03BB207E1F76EDA7CCAA8CF6F
:1000B000CF93DF9360918E00635067FDB7C080914E
:1000C0008B00CCE0D0E0C81BD109CE56DF4F809129
:1000D0008A008D3209F096C0683009F0A5C083EC23
:1000E00080937E008AE5809362001092660088818A
:1000F000807641F0CE01FBD48F3F2FEF920709F4B9
:100100006DC075C09A81109287008981811107C0E6
:100110001092880027E830E082E090E05AC08530F5
:1001200019F490938F0042C08630D1F58B818130D5
:1001300019F488E390E004C0823049F486E290E04C
:1001400090938D0080938C0082E190E025C08330F5
:1001500009F5911109C084E790E090938D00809398
:100160008C0084E090E018C0913049F488E590E07C
:1001700090938D0080938C008CE190E00DC09230C4
:1001800049F48AE490E090938D0080938C008EE097
:1001900090E002C080E090E020E42093660027C059
:1001A000883099F0893039F49093910027E830E055
:1001B00080E090E00EC031E020E08A3009F030E0CD
:1001C000832F922F27E830E004C021E930E081E05E
:1001D00090E030938D0020938C0009C0288127FF88
:1001E00002C08E819F8120E82093660006C02E8188
:1001F0003F812817390708F4C90190936100809363
:10020000600012C08091660087FF0EC0CE0177D7D4
:100210008F3F21F48EE18093620006C0882321F095
:10022000109261001092600010928E008091620026
:1002300084FF62C080916000909161008F3F2FEF3A
:10024000920709F459C0BC018930910510F068E0AB
:1002500070E0861B970B90936100809360009091F3
:100260007E0088E8892780937E00C62F662309F4E4
:100270004EC02091660027FF07C08FE790E041D66F
:10028000C82F893080F521C080918C0090918D001D
:1002900026FF09C0AFE7B0E0FC0124912D93319611
:1002A0006150D9F707C0DC01EFE7F0E02D91219311
:1002B0006150E1F72FEF2C0F30E02F5F3F4F820F9F
:1002C000931F90938D0080938C006C2F8FE790E0AC
:1002D00043D0CC5FCC3071F08FEF9FEF90936100F3
:1002E0008093600007C08FEF9FEF90936100809331
:1002F0006000CEE1C093620084E196B3937069F42C
:100300008150D9F710928F001092890006C060E0EA
:100310008FE790E021D0C4E0DFCFDF91CF91089547
:1003200085B7836085BF8BB780648BBF0895A82F86
:10033000B92F80E090E041E050EA609530E009C0DC
:100340002D9182279795879510F084279527305E09
:10035000C8F36F5FA8F30895EADF8D939D93089526
:10036000CF93CFB7CF93C395B09BE9F7B09B09C0AC
:10037000B09B07C0B09B05C0B09B03C0B09B01C041
:10038000A1C0DF93C0918B00DD27CE56DF4FB09B1D
:1003900002C0DF91EBCF2F930F931F9306B32FEF84
:1003A00000FB20F94F933F9316B34FEF012700FB5B
:1003B00021F93BE031C04E7F012F16B3216028C0E8
:1003C000102F4D7F2260000006B329C04B7F2460B0
:1003D000012F000016B32BC016B3477F28602AC038
:1003E0004F7E06B320612CC04F7D16B320622FC014
:1003F0004F7B06B3206432C0422706B349934FEFC8
:100400000000102710FB20F916B31370C9F1297FE3
:1004100091F2012700FB21F906B3237F89F23150C5
:1004200058F1102710FB22F916B3277E79F2012725
:1004300000FB23F92F7C81F206B3102710FB24F96F
:100440002F7971F200C016B3012700FB25F92F7335
:1004500059F200C006B3102710FB26F9223040F2F3
:1004600000C016B3012700FB27F9243028F64F7788
:10047000206816B30000F9CF10E41ABF002717C098
:100480003B503195C31BD04010E41ABF0881033C98
:10049000E9F00B34D9F0209189001981110F121362
:1004A000EDCF093641F10D3211F0013E39F70093DD
:1004B00090003F914F911F910F912F91DF91CAB7FB
:1004C000C6FD51CFCF91CFBFCF911895209190000D
:1004D000222379F310918E00112311F5343012F19B
:1004E00030938E0020938A0010918B003BE0311BEB
:1004F00030938B0017C000918E0001308CF40AE518
:100500003091620034FD10C000936200CEE7D0E06D
:100510000FC02795A8F45150A9F4220F0000F9CF7D
:100520004AE503C042ED01C0432FC4E1D0E032E010
:1005300017B31360C09A17BB08B320E413E05F93AE
:10054000012756E008BB279520F4515021F4220FD3
:10055000F9CF012756E000003B5A08BBD0F227959F
:1005600028F4515029F4220F0000F9CF012756E05A
:10057000279508BB20F4515021F4220FF9CF012711
:1005800056E02991332308BB21F60C7F10918F0090
:10059000110FC651D04008BB11F01093890010E430
:1005A0001ABF016017B31C7F402F4C7F5F9100C0C2
:1005B00000C008BB17BB48BB7CCF8FB9779BFECF71
:1005C0008FB10895DC01CB0121E1B695A7959795F0
:1005D00087952A95D1F72091AC002817D9F0809300
:1005E000AC00E091A900F091AA008DE40995E0919A
:1005F000A900F091AA0080E00995E091A900F0918E
:10060000AA008091AC000995E091A900F091AA00A0
:1006100080E0099408958091AB008DB98091A80085
:100620008EB90895882319F0883060F101C08AE0FE
:100630002DED32E03093AA002093A9001092A8007B
:1006400091E09093AD008B3071F028F48830B1F0D8
:10065000893091F00AC08C3021F08D3031F480E582
:100660000EC09093A80081E50AC082E58093AB009C
:1006700081E08093A800089582E501C083E580931E
:10068000AB0008952AE633E03093AA002093A90036
:10069000843081F030F4823079F0833079F480E373
:1006A0000EC0863061F020F0873041F483E007C04F
:1006B0008CE005C088E103C080E601C080EC809337
:1006C000AD00089522B79091AD0082B7821B8917C3
:1006D000E0F308951F93CF93DF93182FD8E0C0E085
:1006E00017FF02C0C39A01C0C398110FCC0FB49971
:1006F000CF5FC59AE7DFC598E5DFD15089F78C2F2A
:10070000DF91CF911F91089587B38C6287BBC29808
:10071000C598D8DFC29AD6DFC2988091A90090917F
:10072000AA008D5D924009F476DF1092AC00089526
:1007300087B38C6287BB8091A9009091AA008D5DE0
:10074000924009F468DFC298089587B3837D87BB20
:1007500088B3837D88BB1DB80895CF93DF93C1E232
:10076000C15051F1E091A900F091AA008CEA0995DD
:10077000E091A900F091AA0083E50995E091A90014
:10078000F091AA0080E00995D82FE091A900F0919E
:10079000AA0080E00995D33589F01DB893DFC29A8D
:1007A00091DFC2988FDF8091A9009091AA008D5DA2
:1007B0009240B1F630DFD4CF81E001C080E0DF911C
:1007C000CF910895CF92DF92EF92FF926B017C015F
:1007D000F9DE8C2D8170880F880F880FE091A900B9
:1007E000F091AA0080620995D701C60129E0B6956B
:1007F000A795979587952A95D1F7E091A900F09153
:10080000AA000995D701C601B695A7959795879532
:10081000E091A900F091AA000995E091A900F0915A
:10082000AA0080E0FF90EF90DF90CF900994CF92E4
:10083000DF92EF92FF92CF93DF936B017C01C42F85
:10084000D22FC0DE8C2D8170880F880F880FE09129
:10085000A900F091AA0080640995D701C60129E09A
:10086000B695A795979587952A95D1F7E091A90018
:10087000F091AA000995D701C601B695A79597955D
:100880008795E091A900F091AA000995E091A9004F
:10089000F091AA008C2F0995DD2321F0CF3721F4A8
:1008A0008FE0A6D080E00FC0D2B7CEE1C701B6017D
:1008B00089DF8F37B9F782B78D1B8D33B8F3D2B785
:1008C000C150A1F781E0DF91CF91FF90EF90DF90D1
:1008D000CF900895CF92DF92EF92FF92CF93DF9364
:1008E0006B017C01C42F6EDEE091A900F091AA009B
:1008F0008CE40995D701C60129E0B695A79597958F
:1009000087952A95D1F7E091A900F091AA00099561
:10091000D701C601B695A79597958795E091A9004F
:10092000F091AA000995E091A900F091AA0080E059
:100930000995CF3F19F48FE05BD010C0D2B7CEE15C
:10094000C701B6013FDF8F3F49F482B78D1B8D335E
:10095000B8F3D2B7C150A1F781E001C080E0DF91C8
:10096000CF91FF90EF90DF90CF900895CF93DF93DA
:10097000EC01E091A900F091AA0080EA0995E091CC
:10098000A900F091AA008D2F0995E091A900F0919E
:10099000AA008C2F0995E091A900F091AA0080E0AF
:1009A000DF91CF9109941F93CF93DF93D82F192F05
:1009B000C62FE091A900F091AA0080EC0995E09182
:1009C000A900F091AA00812F0995E091A900F0916A
:1009D000AA008D2F0995E091A900F091AA008C2F13
:1009E00009958EE105D080E0DF91CF911F910895A8
:1009F00090E0981739F032B722B7231B2C33E0F37D
:100A00009F5FF7CF089590E0981739F032B722B77B
:100A1000231B2B3BE0F39F5FF7CF0895BD9ABB9854
:100A2000C39A50E217D05A95E9F70895AC0188E6C9
:100A300005D0842F03D089E601D0852F0FD028E080
:100A400030E0382780FB869506D02A95D1F730FB19
:100A500002D000D06894BB98C39A16F0C398BB9A92
:100A6000E091AE00F091AF003197F0F7C59AE6B390
:100A7000E3FBE091AE00F091AF003197F0F7C5983D
:100A8000089520ECE7DF46F42A95E1F780E02AE1BB
:100A9000E5DF2A95E9F7DECF28E030E0DBDF869559
:100AA00087F938272A95D1F7D5DF27F9322772F34E
:100AB000D1DFD0CFDB01742FB9DF84E2BFDFE1DF0C
:100AC0008D937A95D1F70895DB01742FAFDF83EF13
:100AD000B5DF8DE1B3DF84E6B1DF8D91AFDF82E773
:100AE000ADDFCFDF8078D9F77A9589F70895CF9376
:100AF000DF93EC018981813061F49A9902C085E02D
:100B000002C0809174008EDD10927300A998FCDD04
:100B1000EDC18B3319F48A8176DFE8C1823351F459
:100B20009A9902C085E002C0809174007BDDA9988B
:100B3000FFDDDCC1833359F4C2989A81909364003D
:100B40002E813F8130936E0020936D00BBC18433B2
:100B500061F4C2988A81809364008E819F81909312
:100B60006E0080936D0082E3ADC1863419F4A998BC
:100B700030D4BCC1893411F431D4B8C18A3411F4F1
:100B80003ED4B4C18C3419F48A8147D462C18B3409
:100B900019F48A8162D45DC1873479F48C81813003
:100BA00009F41CD461E08A8182D48E819F81909364
:100BB0006E0080936D0086E385C1883479F40ED48D
:100BC00060E08A8174D48C81809367008E819F81DC
:100BD00090936E0080936D0085E374C18D3579F438
:100BE000C29A8A81809363008C81809368008E8191
:100BF0009F8190936E0080936D008AE363C18C3572
:100C000059F48A81809363008E819F8190936E0056
:100C100080936D0089E356C18E3529F48CD48130E0
:100C200009F0E9C016C18F3511F492D412C1823097
:100C300011F48BDD09C18330F9F4E091A900F09142
:100C4000AA008A81099580937600E091A900F0912D
:100C5000AA008B81099580937700E091A900F0911B
:100C6000AA008C81099580937800E091A900F09109
:100C7000AA008D81099535C18430D1F4809173002B
:100C800081110EC08A819B81092E000CAA0BBB0B1F
:100C900080936F0090937000A0937100B0937200E6
:100CA0008E819F8190936E0080936D0082E00AC1D7
:100CB0008730D1F48091730081110EC08A819B81AD
:100CC000092E000CAA0BBB0B80936F009093700051
:100CD000A0937100B09372008E819F8190936E00FB
:100CE00080936D0083E0EEC08530D9F436DD8093CB
:100CF0007600882309F4AFC0C0917400CC2311F0B2
:100D0000C15001C0C9E0C33008F4A5C08C2F8ADCF3
:100D100024DD80937600C1508111F5CF8C2F82DCC9
:100D20009AC0863079F58091730081110EC08A8156
:100D30009B81092E000CAA0BBB0B80936F00909334
:100D40007000A0937100B09372003C812D81822FBE
:100D50008F7080936A00822F807F40E1849FC00162
:100D60001124830F911D90936C0080936B0020FDE4
:100D7000809369008E819F8190936E0080936D00B7
:100D800081E0A0C0883001F58091730081110EC010
:100D90008A819B81092E000CAA0BBB0B80936F00EC
:100DA00090937000A0937100B093720010926C0049
:100DB00010926B0010926A008E819F8190936E005A
:100DC00080936D0084E07EC0893081F481E080935F
:100DD00073008A819B81AC81BD8180936F00909369
:100DE0007000A0937100B093720080C08A3031F41B
:100DF0008A8180937400109276002DC08B3081F42C
:100E00008A819B819093AF008093AE00C29ABA9A78
:100E100083E0EEDDC298A99880E1EADDFFDD66C0DF
:100E20008C30A1F480EC0ADE80E008DE8AE0E0DDB0
:100E3000C29A85E0DDDDC29885E0DADD87B3837D87
:100E400087BB88B3837D88BBA99A50C08D3031F4AD
:100E500018DE8093760081E090E04AC08E3019F46D
:100E60008A81ECDD43C08F30B1F48A819B81092EE9
:100E7000000CAA0BBB0B80936F0090937000A093A3
:100E80007100B09372008E819F8190936E00809369
:100E90006D0085E017C08031D1F48A819B81092ED5
:100EA000000CAA0BBB0B80936F0090937000A09373
:100EB0007100B09372008E819F8190936E00809339
:100EC0006D0086E0809375008FEF9FEF11C08F3724
:100ED00069F481E0809376009AE190937700109214
:100EE00078008093790084E090E002C080E090E098
:100EF00026E730E030938D0020938C00DF91CF9176
:100F00000895EF92FF920F931F93CF93C62F2091D6
:100F100075003EEF320F323008F494C0253009F4EA
:100F200096C0233339F0293309F460C0263309F021
:100F3000DDC031C020916D0030916E00462F50E031
:100F40002417350708F4C22FF82E8C01802F8F1933
:100F50008C1798F4E091A900F091AA0080E009951F
:100F6000F80181938F0180916D0090916E0001973F
:100F700090936E0080936D00E9CF80916D00909109
:100F80006E00892B09F0B4C080916400882309F4B5
:100F9000AAC0C29AA8C020916D0030916E00462F61
:100FA00050E02417350708F4C22FF82E8C01802F4B
:100FB0008F198C1708F09CC080916D0090916E0085
:100FC000019790936E0080936D00892B41F481E02E
:100FD00044D2F801808313D21092750004C080E0DF
:100FE0003CD2F80180830F5F1F4FE1CF20916D004D
:100FF00030916E00462F50E02417350708F4C22FB9
:10100000F82E8C01802F8F198C1770F480D2F80184
:1010100081938F0180916D0090916E000197909364
:101020006E0080936D00EECF80916D0090916E0008
:10103000892B09F05DC080916300882309F453C0B7
:1010400077D251C08C017C01E60EF11C40C0462FC6
:10105000BC0180916F00909170002CDD80916F0039
:1010600090917000A0917100B09172008C0F911D51
:10107000A11DB11D80936F0090937000A09371002B
:10108000B093720035C080917500823021F5609177
:101090006F0070917000809171009091720092DBEE
:1010A000F801808380916F0090917000A091710091
:1010B000B09172000196A11DB11D80936F009093B5
:1010C0007000A0937100B09372000F5F1F4F0E1558
:1010D0001F05C9F606C080916F009091700046DC34
:1010E000DFCFC83028F41092750002C08FEF01C026
:1010F0008C2FCF911F910F91FF90EF900895EF9259
:10110000FF920F931F93CF93C62F2091750021302C
:1011100031F48C017C01EC0EF11CC0E00BC12430D9
:10112000C1F3263009F4A6C02233B1F12A3309F401
:1011300062C0253309F044C120916D0030916E00EA
:10114000462F50E02417350708F4C22FF82E8C01E3
:10115000802F8F198C1770F4D8018D918D015DD17E
:1011600080916D0090916E00019790936E00809336
:101170006D00EECF80916D0090916E00892B11F083
:1011800080E021C180916700813011F438D101C025
:1011900025D11092750016C120916D0030916E001E
:1011A000462F50E02417350708F4C22FF82E8C0183
:1011B000802F8F198C1790F4E091A900F091AA006C
:1011C000D8018D918D01099580916D0090916E00EF
:1011D000019790936E0080936D00EACF80916D002F
:1011E00090916E00892B61F680916400882309F448
:1011F000E9C0C29AE7C020916D0030916E00462F81
:1012000050E02417350708F4C22FF82E8C01802FE8
:101210008F198C1708F560916800662389F0683093
:1012200030F4F801808149D11092680009C068E06B
:10123000D8018C9142D180916800885080936800D9
:1012400080916D0090916E00019790936E00809355
:101250006D000F5F1F4FDBCF80916D0090916E008E
:10126000892B09F08DCF80916300882309F491CFF9
:101270005FD18FCF462FBC0180916F00909170009D
:1012800023DC80916F0090917000A0917100B0916B
:1012900072008C0F911DA11DB11D80936F00909362
:1012A0007000A0937100B093720080916D009091D6
:1012B0006E008C1B910990936E0080936D00892BBA
:1012C00009F467CF5DCF80917500813009F051C07E
:1012D00020916B0030916C0060916F0070917000F4
:1012E0008091710090917200232B41F521E0F8016B
:1012F00040819DDA80916D0090916E0001979093EE
:101300006E0080936D00892BE1F180916F009091C8
:101310007000A0917100B09172000196A11DB11DE5
:1013200080936F0090937000A0937100B09372004F
:101330000F5F1F4F0E151F0531F640C020E0D8018A
:101340004C9175DA80916900815080936900811118
:10135000D1CF60916F007091700080917100909179
:101360007200F8014081B6DA80916B0080936900C9
:10137000C1CFD8016C9180916F009091700013DB08
:10138000B9CF1092750080916A0081FF15C08091DD
:10139000690090E020916B0030916C0082179307F8
:1013A00059F060916F007091700080917100909180
:1013B0007200F80140818EDAC1E0A7CF8C2F03C004
:1013C0008FEF01C081E0CF911F910F91FF90EF90BF
:1013D0000895C498C398BC98BB980895BB9A84E1BB
:1013E0008A95F1F7BC9884E18A95F1F7BB9884E17E
:1013F0008A95F1F7BC9A84E18A95F1F70895BB9A32
:10140000BC9A84E18A95F1F7BB9884E18A95F1F75B
:10141000BC9884E18A95F1F7089598E0BB9A87FF1C
:1014200002C0BC9801C0BC9A24E12A95F1F7BB9890
:1014300024E12A95F1F7880F915081F7BB9ABC9867
:1014400084E18A95F1F7BB9824E12A95F1F786B3F8
:101450008295817091E089270895282FBB9ABC98C6
:1014600034E13A95F1F7BB9884E18A95F1F796B3A8
:1014700094FB882780F997E0BB9A34E13A95F1F71D
:10148000BB9834E13A95F1F7880FB4998160915097
:1014900099F7BB9A211102C0BC9A01C0BC9894E193
:1014A0009A95F1F7BB9834E13A95F1F708956130D8
:1014B00011F4816001C08E7FB0CFEF92FF920F9345
:1014C0001F93CF93DF9307E010E0061B1109C7E0DD
:1014D000D0E0E82EF12CC017D10791F0C7010C2EF7
:1014E00002C0959587950A94E2F780FF02C0C39ADF
:1014F00001C0C398C59AE6D8C598E4D82197EBCF28
:10150000DF91CF911F910F91FF90EF900895CF93AE
:10151000DF93D8E0C0E0CC0FC59AD4D8C598D2D814
:10152000B499CF5FD150B9F78C2FDF91CF91089547
:10153000C298C598C7C8C29A88E28A95F1F7C2D8FE
:10154000B49B03C0C29880E00895C29881E00895DA
:10155000CF93C29A88E28A95F1F7B4D868E080EC1C
:10156000ACDFC0E0C59AAED8B49904C0CA5FC598D4
:10157000A9D806C0C598A6D8CF5FC83099F7CFEFD5
:10158000C2988C2FCF91089512BA18BA11BA8FEF62
:1015900087BB17BA83E084BB9EEF95BB83BFC0D6E1
:0A15A000789486D5FECFF894FFCFB3
:0615AA00FFFF5A010100E1
:00000001FF
